:1000000009C016C015C014C013C012C011C010C062
:1000100099C00EC011241FBECFE9CDBF10E0A0E6ED
:10002000B0E001C01D92A239B107E1F7CBD0CCC13D
:10003000E7CF20916600922F9F5F9F71909366009B
:100040009EBB8DBB84E28CBB86E28CBBE199FECF6C
:100050002EBB84E18CBB86E18CBB089540E250E06E
:1000600060E070E082E790E0A0D18091660001C07E
:100070008F5FE82FF0E0EE58FF4F90819F3F19F41B
:100080008032B0F307C080936600803218F49093FA
:1000900064000895109266000895809164008111B3
:1000A0000CC08091620090916300019631F48091C0
:1000B0006100815080936400089580916400909164
:1000C0006200890F80936400809164002091610038
:1000D00030E090E08217930714F0109264000895C6
:1000E000F894A89581B5886181BD85E481BD789437
:1000F0000895F894A89584B7877F84BF81B58861F7
:1001000081BD11BC7894089581E687B9A29A86ECE6
:1001100086B9089537980895369A3699FECF95B1E5
:10012000981760F4809160008F5F893018F4809395
:10013000600006C01092600081E008951092600097
:1001400080E008951F920F920FB60F9211242F9303
:100150003F934F935F936F937F938F939F93AF934F
:10016000BF93EF93FF93809167008F3F19F08F5FEC
:100170008093670080916700823099F480916500D8
:10018000882319F0809164000BC0809162009091E7
:100190006300019721F080916100815001C080E0EF
:1001A00048DFFF91EF91BF91AF919F918F917F9128
:1001B0006F915F914F913F912F910F900FBE0F90D4
:1001C0001F90189589E188BB82E087BB83E28FBDD1
:1001D00081E083BF99DF479A80916100E82FF0E0CA
:1001E000E859FF4F98E09083E82FEF5FF0E0E8597F
:1001F000FF4F9EE09083E82FEE5FF0E0E859FF4F5D
:1002000097E29083E82FED5FF0E0E859FF4F98E721
:1002100090838C5F8093610081E090E09093630015
:10022000809362001092650085B7877E85BF16DFD8
:100230008091640084FF06C0809164008F70809379
:1002400064002BDF809164008061F3DE49DFE09180
:100250006400F0E0E859FF4F808189BD82E85CDFEF
:10026000882309F49AC080916400811135C099B542
:10027000E0916400F0E0E859FF4F8081891760F158
:1002800088E74ADF8823E1F38BE015C02FE739EADE
:1002900093E0215030409040E1F700C00000909181
:1002A000680099BD2FEF32E597E021503040904033
:1002B000E1F700C00000815019BC8111E7CF19DFC0
:1002C00085B7877E806185BF85B7806285BF889549
:1002D00085B78F7D85BF58C089B519BC2FE739EA2E
:1002E00093E0215030409040E1F700C0000089BD0C
:1002F0002FEF32E597E0215030409040E1F700C009
:10030000000019BC2FE739EA93E0215030409040BB
:10031000E1F700C0000089BD2FEF32E597E02150E2
:1003200030409040E1F700C0000019BC2FE739EAE7
:1003300093E0215030409040E1F700C0000089BDBB
:100340002FEF32E587E0215030408040E1F700C0D8
:10035000000089B5909168008695891720F499BDB1
:100360001092640003C089B5869589BD99B5E09166
:100370006400F0E0E859FF4F8081981728F48091DD
:1003800064008150809364009FEF21EF3BE2915025
:1003900020403040E1F700C0000085B7806285BF93
:1003A000889585B78F7D85BF59CFA82F862FE82FD9
:1003B000E199FECF1FBA05C0EEBBE09AE3950DB2FE
:0C03C0000D924150C8F70895F894FFCF4B
:00000001FF
